:100000000C941E060C94BA270C94E7270C94460611
:100010000C9446060C94DC120C9446060C9446068E
:100020000C9446060C9446060C9446060C94460620
:100030000C9446060C9446060C9446060C94460610
:100040000C9414280C9446060C94022C0C94452C09
:100050000C9446060C9446060C9446060C944606F0
:100060000C9446060C9446064518A718861889185D
:100070008C188F18921895189818A718A118D919C4
:10008000DB19DB19D919DB19DB19DB19DB19DB19D2
:10009000DB19DB19DB19DB19DB19DB19DB19DB19C0
:1000A0005F19DB19DB19DB19DB19DB19D018DB1938
:1000B000DB19DB19DB19DB19DB19DB19DB19DB19A0
:1000C000DB19DB19DB19DB19DB19DB196B196B1970
:1000D0006B196B196B196B196B196B196B19DB1990
:1000E000DB19DB19DB19DB19DB19D0186A196A195E
:1000F0006A196A19DB1978197E1984198A199019F5
:1001000096199C19A219AC19B619C019CA19111956
:10011000D318DB19DB19DB19DB195F19DB19DB19C4
:10012000DB19DB19DB19DB19DB19DB196919691913
:1001300069196919DB1978197E1984198A199019B6
:1001400096199C19A219AC19B619C019CA19111916
:10015000D318DB19DB19DB19DB195F190E1A0E1A1C
:100160000E1A0E1A0E1A0E1A0E1A0E1A0E1A0E1A4F
:100170000E1A0E1A0E1A241B241B241B241B241BCC
:10018000241B531A5D1A671A711ACE1AD81AE71A65
:10019000F81A801C951CA11CAA1CB91CDE1CE71CAB
:1001A000301DF91C432049204F2056206420862012
:1001B000A420456E746572206D656E752E2E2E001E
:1001C000546F67676C6564206D6963726F50504D42
:1001D00000546F67676C656420696E76657274653C
:1001E000642050504D2100546F67676C6564205443
:1001F00058206D7574696E672100546F67676C6570
:10020000642074656C656D65747279210050726F3D
:10021000746F636F6C206572726F72207769746897
:100220002052580054696D656F7574207768656E4B
:1002300020636F6E6E656374696E6720746F205201
:100240005800507265737320616E79206B65792058
:10025000746F2063616E63656C00436F6E6E6563DF
:1002600074696E6720746F2052582C20706F776508
:100270007220757020746865205258202877697440
:10028000682062696E6420706C7567206966206EF4
:100290006F74207573696E6720616C776179732064
:1002A00062696E642900546F67676C656420276912
:1002B0006D6D656469617465206F75747075742700
:1002C00000546F67676C65642027736C61766520E6
:1002D0006D6F64652700546F67676C6564202761E4
:1002E0006C776179732062696E642700546F676769
:1002F0006C65642050504D206368616E6E656C20A3
:100300006C696D69740053657420525353492069B8
:100310006E6A656374696F6E206368616E6E656C8A
:100320002028303D3D64697361626C652900536526
:10033000742050504D206D696E696D756D20737914
:100340006E630053657420626561636F6E20696E31
:1003500074657276616C0053657420626561636FC9
:100360006E2064656C617900536574206265616319
:100370006F6E206672657175656E637920696E2097
:10038000487A3A20303D64697361626C652C205074
:10039000783D504D52206368616E6E656C20782CFC
:1003A0002046783D465253206368616E6E656C202E
:1003B00078005365742050574D2073746F7020641B
:1003C000656C61792028302064697361626C6564B2
:1003D0002C20312D323535203D3D20302E317320FB
:1003E0002D2035306D696E29005365742050504DB5
:1003F0002073746F702064656C61792028302064EC
:10040000697361626C65642C20312D323535203D75
:100410003D20302E3173202D2035306D696E29003E
:10042000536574206661696C736166652064656CF0
:1004300061792028302064697361626C65642C20C6
:10044000312D323535203D3D20302E3173202D2089
:1004500035306D696E29002A2A2A2A2A2A2A2A2A50
:100460002A2A2A2A2A2A2A2A2A2A2A2A2A2A2A2AEC
:100470002A2A2A2A0052582041636B6564202D20C5
:1004800072657665727420737563636573736675E0
:100490006C21002A2A2A2A2A2A2A2A2A2A2A2A2AAD
:1004A0002A2A2A2A2A2A2A2A2A2A2A2A2A2A2A2AAC
:1004B000002A2A2A2A2A2A2A2A2A2A2A2A2A2A2AC6
:1004C0002A2A2A2A2A2A2A2A2A2A2A2A2A2A00528E
:1004D000582041636B6564202D20757064617465DC
:1004E000207375636365737366756C21002A2A2A0D
:1004F0002A2A2A2A2A2A2A2A2A2A2A2A2A2A2A2A5C
:100500002A2A2A2A2A2A2A2A2A2A0056616C696457
:100510002063686F69636573206172653A205B319F
:100520005D2D5B31365D20286368616E6E656C20E1
:10053000312D31362900536574206F7574707574D0
:1005400020666F7220706F727420005B585D2061AE
:10055000626F7274206368616E67657320616E6498
:10056000206578697420525820636F6E6669670051
:100570005B535D20736176652073657474696E6783
:100580007320746F205258005B525D20726576654F
:1005900072742052582073657474696E6773207486
:1005A0006F2064656661756C747300557365206EA9
:1005B000756D62657273205B312D445D20746F2010
:1005C0006564697420706F727473205B452D515D92
:1005D00020666F722073657474696E677300202DD6
:1005E00020726563656976657220636F6E66696700
:1005F000757261746F722C20727820737720000AF4
:100600000A6F70656E4C52536E67200053657420FC
:1006100073657269616C2062617564726174653AB8
:10062000200056616C69642063686F696365733A82
:100630002031202D20342B34202F2032202D203823
:10064000202F2033202D20382B34202F2034202D14
:10065000203132202F2035202D2031322B34202FF5
:100660002036202D20313600536574204368616E9A
:100670006E656C20636F6E6669673A20005365741F
:100680002044617461726174652028302D32293AEA
:10069000200053657420486F70206368616E6E653A
:1006A0006C7320286D61782032342C207365706162
:1006B000726174656420627920636F6D6D61732966
:1006C0002076616C69642076616C75657320312DCC
:1006D0003235353A2000536574206368616E6E656B
:1006E0006C2073706163696E6720287831306B48C5
:1006F0007A293A200053657420524620706F77653E
:10070000722028302D37293A200053657420524634
:10071000206D6167696320286865782920652E67E8
:100720002E20307844454144463030443A2000532E
:1007300065742062617365206672657175656E63AC
:10074000792028696E20487A293A20005B5A5D207A
:10075000656E746572207265636569766572206383
:100760006F6E66696775726174696F6E2075746902
:100770006C79005B465D20646973706C61792061FF
:10078000637475616C206672657175656E63696509
:10079000732075736564005B525D2063616C6375E3
:1007A0006C6174652072616E646F6D206B65792079
:1007B000616E6420686F70206C697374005B495DC2
:1007C000207265696E697469616C697A6520736508
:1007D0007474696E677320746F20736B65746368DB
:1007E0002064656661756C7473005B585D2072658A
:1007F00076657274206368616E67657320616E64EC
:100800002065786974206D656E75005B535D20739B
:100810006176652073657474696E677320746F20E8
:10082000454550524F4D20616E64206578697420B3
:100830006D656E7500557365206E756D62657273BA
:10084000205B302D395D20746F20656469742070E1
:100850006172616D657465727300202D2053797328
:1008600074656D20636F6E66696775726174696F18
:100870006E000A0A6F70656E4C52536E672000510D
:1008800029204F7574707574206265666F726520DB
:100890006C696E6B20283D465329203A2000502970
:1008A00020536C617665206D6F64652028657870D3
:1008B0006572696D656E74616C293A20004F29205C
:1008C00054696D65642042494E44206174207374FC
:1008D000617274757020203A20004E292050504DCE
:1008E000206F7574707574206C696D69746564200F
:1008F000202020203A200044495341424C454400E6
:100900004D292050504D205253534920746F20637D
:1009100068616E6E656C202020203A20004C2920F2
:1009200050504D206D696E696D756D2073796E63E1
:10093000202875732920203A200044495341424C15
:100940004544004B29204661696C736166652062ED
:100950006561636F6E20696E74762E2028312D32AA
:10096000353573293A20004A29204661696C736144
:10097000666520626561636F6E2064656C617920D5
:1009800028302D323535203D3E20313073202D204A
:100990003135306D696E293A200049292046616958
:1009A0006C7361666520626561636F6E206672714B
:1009B0002E203A200048292050574D2073746F7024
:1009C0002064656C6179202020202020203A2000BE
:1009D00047292050504D2073746F702064656C61FE
:1009E00079202020202020203A200046292046611E
:1009F000696C736166652064656C617920202020D4
:100A00002020203A200050574D206368616E6E65AB
:100A10006C200066756E6374696F6E3A2000292041
:100A2000706F72742000506F776572546F776572C3
:100A300000445446205548462033322D62697420C4
:100A400031306368004F70656E4C52536E67525878
:100A5000206D696E6920342F36636800466C7974A6
:100A6000726F6E2F4F72616E6765525820554846FF
:100A70002038636800525820747970653A20004429
:100A8000697361626C656400487A00203D3D200016
:100A900043616C63756C61746564207061636B6540
:100AA0007420696E74657276616C3A200042292068
:100AB0004D6963726F202868616C66292050504D23
:100AC000202020203A00412920496E766572746505
:100AD000642050504D20696E20202020203A0030A4
:100AE00029204D7574652062757A7A657220286DAB
:100AF0006F73746C79293A003929205365726961E2
:100B00006C2062617564726174653A00736D617224
:100B100074506F7274004672536B79005472616E38
:100B200073706172656E740044697361626C6564B0
:100B30000038292054656C656D657472793A2020FF
:100B40002020202020003729204368616E6E656CCC
:100B500020636F6E6669673A202000362920446161
:100B60007461726174652028302D32293A2020206A
:100B700000352920486F70206368616E6E656C7364
:100B80003A2020202020003429204368616E6E65C1
:100B90006C2073706163696E673A202000332920EE
:100BA000524620706F7765722028302D37293A2001
:100BB0002020003229205246206D616769633A2067
:100BC0002020202020202020003129204261736530
:100BD000206672657175656E63793A202020000089
:100BE00000000700020100000304060000000000EE
:100BF00000000001020408102040800102040810D7
:100C00002001020408102004040404040404040263
:100C10000202020202030303030303000000002395
:100C2000002600290000000000250028002B0000FD
:100C3000000000240027002A0000332D11241FBECD
:100C4000CFEFD8E0DEBFCDBF13E0A0E0B1E0E4E736
:100C5000F0E602C005900D92A83CB107D9F716E066
:100C6000A8ECB3E001C01D92AC38B107E1F71CE07D
:100C7000CCE3DCE004C02297FE010E943C2ECA3384
:100C8000D107C9F70E946F2D0C9438300C940000E6
:100C900080917105813019F482E080937105809113
:100CA0007105833019F484E0809371050895A89547
:100CB0000895DC01ED91FC910190F081E02D099502
:100CC00008952091720530917305382748E0C901D5
:100CD000880F991F37FF06C09C0151E2252750E17C
:100CE000352701C09C01415091F730937305209343
:100CF0007205089588E38093740580E092ECA1E08A
:100D0000B0E08093750590937605A0937705B09336
:100D1000780587E08093810580E091EAACEBB3E34E
:100D20008093790590937A05A0937B05B0937C0519
:100D300085E0809382058DEE9EEFADEABEED809357
:100D40007D0590937E05A0937F05B0938005E3E831
:100D5000F5E080E090E0863028F4DC01AE54BC4F32
:100D60002C9101C020E0219301968831910599F7DB
:100D700082E080939B058AE080939C05089580E043
:100D80009EECADEEB4E38093B9059093BA05A093C1
:100D9000BB05B093BC0580E090E0A0E0B0E5809397
:100DA000BD059093BE05A093BF05B093C005E1ECCF
:100DB000F5E080E081938F5F8031E1F70895A0E056
:100DC000B0E0E5EEF6E00C94052ED82F0E946A28DC
:100DD0006115710581059105C9F30E94A82E109235
:100DE0007D0510927E0510927F0510928005C4E06B
:100DF000812C912C54018A94C0907D05D0907E0561
:100E0000E0907F05F0908005FE2CED2CDC2CCC24AE
:100E10000E94A32EA50194010E94E42D6C0D7D1D5E
:100E20008E1D9F1D60937D0570937E0580937F05C9
:100E300090938005C15001F7DD2309F450C003E809
:100E400015E0E801A12CB12C62E3C62ED12CE12CD7
:100E5000F12C8881882309F442C0B39419F40E94CC
:100E60007A063DC00E94A32EA70196010E94E42DA0
:100E7000E1E0E60FA3E8B5E08A2F801B8A1520F495
:100E80008D918E13F9CFE9CF2091820530E0A0E15A
:100E9000B7E20E947C2D9B01AC01AE2FB0E00E9416
:100EA0008B2D4090790550907A0560907B0570906D
:100EB0007C05640D751D861D971D4090B9055090E9
:100EC000BA056090BB057090BC05461657066806CB
:100ED000790618F2E993A39488E1A812BACFCDB7A6
:100EE000DEB7E0E10C94212E8436910520F4BC019C
:100EF00080E090E017C09C018E3B910528F42A55B4
:100F00003109AAE0B0E00CC0823D910528F4245BD1
:100F10003109A4E6B0E004C02D5C3109A8E5B2E0D7
:100F20000E947C2DA4E6B0E09B01AC010E948B2DB9
:100F3000089590E08C599F4F0E947407089561E0D6
:100F40008AE00E94172960E08AE00E9450290895F3
:100F5000892B11F061E001C060E08AE00E94502915
:100F6000089560E089E00E94172961E088E00E940E
:100F7000172961E087E00E94172960E082E00E9463
:100F8000172961E084E00E941729089542E050E0AB
:100F900068E476E080E00E949A270895E3E0F0E0BC
:100FA00089E080935700E491E67081E0E63009F033
:100FB00080E00895CF93DF93C82F0E94CE07882347
:100FC00081F0DFB781E080937005F8940E945706A6
:100FD00088E180936000C0936000C1110E945706B1
:100FE000DFBFDF91CF9108958F929F92AF92BF9212
:100FF000CF92DF92EF92FF92CF93FC01C0A5EC2F2E
:10100000E770F0E0E658FC4FA081B0E0C7FF03C0F6
:1010100024E130E002C02FE030E0FC0197A183E141
:10102000989FF0011124E25CFE4F80809180A280A5
:10103000B380A20FB31F20E43FE14DE750E00E94D0
:10104000962DA50194010E94C22D8C2F887149F420
:1010500069017A01E0EDCE0EE7E0DE1EE11CF11C35
:101060001BC0C7FF05C060E47AE88CE29EE004C0C4
:1010700060E07EEE8AEB9BE069017A01F8EBCF0E2F
:10108000FBE0DF1EE11CF11CA50194010E94C22DB2
:10109000C20ED31EE41EF51EC701B60169517C4F76
:1010A0008F4F9F4F28EE33E040E050E00E94C22D6A
:1010B000A8EEB3E00E948B2DCF91FF90EF90DF90D0
:1010C000CF90BF90AF909F908F9008958F3F9105E4
:1010D00051F048F0811522E0920738F081159340D5
:1010E00030F482E0089580E0089581E0089583E07F
:1010F0000895A0E0B0E0EFE7F8E00C940E2EEB01CD
:101100008A01B82FB695A0E028813981F8012083A3
:101110002A813B8121832C813D8122832E813F8145
:101120002383688179814A815B812C813D81EE81B5
:10113000FF819F2F9295990F990F907C272F2370F5
:10114000922B252F2370220F220F922B232F2370F7
:101150002295207F922BF80194830B5F1F4F2896D6
:10116000AF5FBA1788F680FF24C0888199810E94FA
:101170006608D82E8A819B810E946608E82E8C81A1
:101180009D810E946608F82E8E819F810E946608CC
:10119000F0E4DF9EA001112490E1E99E900111246A
:1011A000242B282BE4E0FE9EB0011124262BF8010D
:1011B0002083CDB7DEB7E7E00C942A2E803223E0FF
:1011C000920708F1883E23E0920740F48F51934044
:1011D000E4E096958795EA95E1F70895803D27E04C
:1011E000920718F48C5D93400895883928E092079F
:1011F00068F4885C974074E0969587957A95E1F756
:101200008D509C4F089580E090E008958FEF93E01B
:1012100008958C30910540F4A4E0880F991FAA9599
:10122000E1F7885D9C4F0895843F23E0920718F40E
:1012300084529C4F0895811524E0920740F486570C
:10124000934FF4E0880F991FFA95E1F7089580E92C
:1012500098E008959C013695279525753575821B74
:10126000930B9C0123733373969587959695879579
:1012700083739373820F931F9C0154E036952795D7
:101280005A95E1F7280F391F2F703F7041E051E068
:10129000249FC001259F900D349F900D1124892F0C
:1012A00008955F98882319F00000289A02C0000072
:1012B000289800005F9A000008955F9A000083B1AB
:1012C0005F980000869581700895CF93DF93D82FA3
:1012D0005C9A5F985C98C8E08D2F80780E945109D5
:1012E000DD0FC150C9F75F98DF91CF9108958F77D7
:1012F0000E9465090895CF93DF93D82FC8E08D2F02
:1013000080780E945109DD0FC150C9F75F98DF91C5
:10131000CF910895CF93DF935F98C8E080E0D82FF6
:10132000DD0F0E945D098D0FC150C9F7DF91CF918C
:1013300008950E9477090E948A095C9A0895A1E0A5
:10134000B0E0E5EAF9E00C94132E806869830E940E
:1013500065096981862F0E947B095C9A2196E2E0EB
:101360000C942F2ECF93C0917D05C827E82FF0E075
:10137000EC58FA4F678589E70E949F096C2F8DE32F
:101380000E949F096C2F82E40E949F09CF910895CB
:1013900086E20E9499090895CF93DF93EC016C8156
:1013A0008CE10E949F096D818DE10E949F096E81F1
:1013B0008EE10E949F096F8180E20E949F096885EB
:1013C00081E20E949F09698582E20E949F096A85E5
:1013D00083E20E949F096B8584E20E949F096C85CD
:1013E00085E20E949F096D858AE20E949F096E85B1
:1013F0008EE60E949F096F858FE60E949F0968898B
:1014000080E70E949F09698981E70E949F096A8994
:1014100082E70E949F09DF91CF910895CF92DF92DA
:10142000EF92FF92CF93DF936B017C01C11488E3AD
:10143000D8068CE9E8068CE1F80628F5C701B60164
:1014400020E836E948E950E00E94C22DE90168979A
:1014500060E879E687E69FEF0E949E2D6C0D7D1D6A
:101460008E1D9F1DF2E0660F771F881F991FFA954A
:10147000D1F721E732E040E050E00E94C22DF22E89
:10148000E32E80E421C0C701B60120E03DE241E344
:1014900051E00E94C22DE901689760E073ED8EEC87
:1014A0009EEF0E949E2D6C0D7D1D8E1D9F1D660F53
:1014B000771F881F991F21E732E040E050E00E942B
:1014C000C22DF22EE32E80E66C2F6F71680F85E738
:1014D0000E949F096E2D86E70E949F096F2D87E766
:1014E0000E949F09DF91CF91FF90EF90DF90CF9006
:1014F0000895682F8DE60E949F0908958F929F920C
:10150000AF92BF92CF92DF92EF92FF92CF93DF9391
:10151000D82F83E00E94990980936F0584E00E9490
:10152000990980936E0560E086E00E949F0961E062
:1015300087E00E949F096FE789E00E949F0965E0AC
:101540008AE00E949F0962E18BE00E949F0965E1A9
:101550008CE00E949F096DEF8DE00E949F0960E082
:101560008EE00E949F09DD2319F08BE291E008C014
:1015700020919B0533E1239FC0011124825C9E4F83
:101580000E94CC096CE880E30E949F096FE082E32F
:101590000E949F0962E483E30E949F0980919C0559
:1015A00087FF02C064E101C06AE084E30E949F09F2
:1015B0006AE285E30E949F096DE286E30E949F092B
:1015C00064ED87E30E949F0960E088E30E949F0921
:1015D00060E089E30E949F09D11109C0C0907D0598
:1015E000D0907E05E0907F05F090800507C0C5E9AA
:1015F000CC2EC1ECDC2EED2CCEEDFC2ECAE38F2CD4
:101600009924AA24BB24682D8C2F0E949F09682D41
:1016100085E08C0F0E949F09FE2CED2CDC2CCC2445
:10162000CF5FCE3361F76FEF83E40E949F096FEFC6
:1016300084E40E949F096FEF85E40E949F096FEF89
:1016400086E40E949F09DD2311F066E002C06091EC
:1016500081058DE60E949F0960E089E70E949F094D
:10166000609182058AE70E949F0960E083E70E94FB
:101670009F0960E084E70E949F09D11109C0609131
:10168000790570917A0580917B0590917C0504C065
:1016900060E071EA8CEB93E30E940E0ADF91CF9138
:1016A000FF90EF90DF90CF90BF90AF909F908F9082
:1016B000089561E087E00E949F0964E28EE70E943E
:1016C0009F0963E088E00E949F0960E088E00E9433
:1016D0009F0965E087E00E949F0962E085E00E9423
:1016E0009F0983E00E94990980936F0584E00E941E
:1016F000990980936E05089583E00E94990980936B
:101700006F0584E00E94990980936E0561E087E08F
:101710000E949F096AE070E080E090E00E948D28BE
:101720000E94590B00000895CF92DF92FF920F9311
:101730001F93CF93DF931F92CDB7DEB7082F162FDD
:101740008EE399830E949F09F02EC02E9981D92E95
:101750008C2D8F19811738F4F60161916F018FE795
:101760000E949F09F5CF64E085E00E949F0983E015
:101770000E94990980936F0584E00E9499098093E3
:101780006E050E946A2860936A0570936B058093CA
:101790006C0590936D0569E087E00E949F0981E0E8
:1017A000809371050F90DF91CF911F910F91FF9062
:1017B000DF90CF9008950F931F930E94940B809118
:1017C0007105813099F40E946A2800916A05109190
:1017D0006B0520916C0530916D05601B710B820BC0
:1017E000930B603A76488140910548F380917105EA
:1017F000813031F46EE971E080EE95E00E94562A66
:101800001F910F9108950F931F938091710582305E
:1018100021F41092710581E020C080917105813022
:10182000D9F40E946A2800916A0510916B052091F5
:101830006C0530916D05601B710B820B930B613A47
:1018400076488140910540F061E087E00E949F0961
:101850001092710582E001C080E01F910F91089500
:10186000CF93DF93EC014AE050E06D2F70E080EE03
:1018700095E00E94242B6EE280EE95E00E94282ADB
:10188000BE0184E0769567958A95E1F76F707727BA
:101890004AE050E080EE95E00E94242BDF91CF914A
:1018A0000895D82FC0E0CD1780F42D9A64E670E03B
:1018B00080E090E00E948D282D9864E670E080E042
:1018C00090E00E948D28CF5FEECF6CE271E080E067
:1018D00090E00E948D28E6CF0F931F93CF93DF9364
:1018E000EC01062F15E0115051F0CE010E941F307F
:1018F000081741F0602FCE010E942730F4CF82E01C
:101900000E94510CDF91CF911F910F910895A0E09B
:10191000B0E0EDE8FCE00C94052E482E562EC0E019
:10192000D0E0612C712CE12CF12C00E010E0411092
:101930000CC06090D20586E4689E3001112459E104
:10194000E52EF12C08EB15E01EC091E049120FC006
:101950006090D205E6E46E9E30011124FBE16F0E2B
:10196000711C49E2E42EF12C04E715E00CC082E082
:10197000481209C028E1622E77247394EE24E39480
:10198000F12C01ED15E043018C0E9D1E10927305A4
:10199000109272053401A62CA818B12CC30101962F
:1019A0006C01AE14BF04A8F4A00EB11E511006C005
:1019B000C3010E941F30F501808305C0F5016081DD
:1019C000C3010E946C0CF50180810E946106360102
:1019D000E2CFC301511018C0C3010E941F30B82EBE
:1019E000C6010E941F302B2D30E0322F2227282BDA
:1019F00080917205909173058217930779F4C0E086
:101A0000D0E05524539493CF3601609173050E9422
:101A10006C0C60917205C6010E946C0CC05EDE4FBA
:101A2000C13E92E0D90708F482CF852DCDB7DEB74D
:101A3000E0E10C94212E61E082E00E94870C089581
:101A400060E082E00E94870C8091D105853028F00B
:101A500084E08093D1050E941B0D8091D105809375
:101A6000D205089561E080E00E94870C61E081E08A
:101A70000E94870C089560E080E00E94870C882314
:101A800051F060E081E00E94870C882321F0809172
:101A90007405883349F00E94BF060E947A0681E0EF
:101AA0000E94DF060E94320D0895882319F06AEA29
:101AB00071E002C06EEA71E080EE95E00E94562A65
:101AC0000895FF920F931F93CF93DF9369EC7BE010
:101AD00080EE95E00E94022A4091790550917A05A6
:101AE00060917B0570917C052AE030E080EE95E006
:101AF0000E942B2B63EB7BE080EE95E00E94022A94
:101B000040917D0550917E0560917F057091800523
:101B100020E130E080EE95E00E942B2B6DE97BE028
:101B200080EE95E00E94022A4AE050E06091810533
:101B300080EE95E00E94532B67E87BE080EE95E015
:101B40000E94022A4AE050E06091820580EE95E012
:101B50000E94532B61E77BE080EE95E00E94022A11
:101B6000C3E8D5E0F12C8E0188818823A9F0FF20FD
:101B700031F061EB71E080EE95E00E94252A21961C
:101B80004AE050E0F801608180EE95E00E941C2B55
:101B9000F394F8E1FF12E7CF80EE95E00E94302A3F
:101BA0006BE57BE080EE95E00E94022A4AE050E07F
:101BB00060919B0580EE95E00E94532B66E47BE0EC
:101BC00080EE95E00E94022AE0919C05E770F0E02B
:101BD000EE0FFF1FEE57FC4F6081718180EE95E0A4
:101BE0000E94562A61E37BE080EE95E00E94022A83
:101BF00080919C058871883069F028F4811113C0A8
:101C000068E27BE00CC0803141F0883161F46CE027
:101C10007BE005C06CE17BE002C066E17BE080EE2A
:101C200095E00E94442A68EF7AE080EE95E00E94F9
:101C3000022A409175055091760560917705709163
:101C400078052AE030E080EE95E00E942B2B6FEDC6
:101C50007AE080EE95E00E94022A8091BD058071B5
:101C60000E94550D66EC7AE080EE95E00E94022A13
:101C70008091BD0580740E94550D6DEA7AE080EE7A
:101C800095E00E94022A8091BD0580720E94550D48
:101C900060E97AE080EE95E00E94022A84E795E010
:101CA0000E94F407AB01BC012AE030E080EE95E031
:101CB0000E940D2B6BE87AE080EE95E00E94022AEC
:101CC00084E795E00E94F4079B01AC0160E472E4B4
:101CD0008FE090E00E94C22DBA01A9012AE030E015
:101CE00080EE95E00E940D2B68E87AE080EE95E0AA
:101CF0000E94442ACDB7DEB7E5E00C942C2E8F92DB
:101D00009F92AF92BF92CF92DF92EF92FF9281119A
:101D100007C06FE77AE080EE95E00E94442A2FC06A
:101D200090E00E94740724E630E040E050E00E941A
:101D3000C22DCA01B9012AE030E040E050E00E9423
:101D4000C22D49015A016B017C012AE030E0B50146
:101D5000A40180EE95E00E940D2B6EE280EE95E0EE
:101D60000E94282A2AE030E0B701A60180EE95E023
:101D70000E940D2B63E780EE95E00E94682AFF9099
:101D8000EF90DF90CF90BF90AF909F908F9008958D
:101D90001F93CF93DF9365E77AE080EE95E00E9492
:101DA000022A80919D05813041F46CE57AE080EE55
:101DB00095E00E94442A10E050C0823019F465E496
:101DC0007AE0F5CF843019F461E37AE0F0CF853022
:101DD00091F766E27AE0EBCFC12FD0E0C930D105B0
:101DE0000CF441C068E3610F80EE95E00E94282A60
:101DF0006EE17AE080EE95E00E94022ABE016F5FFC
:101E00007F4F4AE050E080EE95E00E94EC2A63E1CB
:101E10007AE080EE95E00E94022AC356DA4FE9810B
:101E2000E03218F566E07AE080EE95E00E94022A42
:101E30008981803130F06DE673E080EE95E00E949C
:101E4000252A69816F7070E06F5F7F4F4AE050E034
:101E500080EE95E00E94F52A1F5F809146051817D5
:101E600008F4BACF0FC061E3BECFEF70F0E0EE0F21
:101E7000FF1FEE56FC4F6081718180EE95E00E945D
:101E8000562AEACF6BEE79E080EE95E00E94022AB6
:101E90008091B5050E947F0E60ED79E080EE95E0BF
:101EA0000E94022A8091B6050E947F0E65EB79E0C0
:101EB00080EE95E00E94022A8091B7050E947F0E75
:101EC0006AE979E080EE95E00E94022A4091AD0532
:101ED0005091AE056091AF057091B0054115510567
:101EE0006105710539F12AE030E080EE95E00E944D
:101EF0002B2B67E679E080EE95E00E94022A809124
:101F0000B1050E949907AB01BC012AE030E080EEE8
:101F100095E00E942B2B63E479E080EE95E00E942F
:101F2000022A4AE050E06091B20580EE95E00E94FE
:101F3000532B06C06AE379E080EE95E00E94442AC4
:101F40006DE179E080EE95E00E94022A6091B30590
:101F50007091B4054AE050E080EE95E00E943D2B80
:101F600060E079E080EE95E00E94022A6091AC0585
:101F7000603450F470E06F5F7F4F4AE050E080EED5
:101F800095E00E94F52A06C067EF78E080EE95E0C4
:101F90000E94442A6AED78E080EE95E00E94022AD1
:101FA0008091AB0580FF03C063EB71E002C067EB7B
:101FB00071E080EE95E00E94562A6DEB78E080EEAD
:101FC00095E00E94022A8091AB0582700E94550D17
:101FD0006EE978E080EE95E00E94022A8091AB05E0
:101FE00084700E94550D6FE778E080EE95E00E94C6
:101FF000022A8091AB0588700E94550DDF91CF9128
:102000001F9108950F931F93CF93DF932091430562
:102010002F3FA9F56FEF75E080EE95E00E94022A50
:1020200080E893E00E94300C6EED75E080EE95E064
:102030000E94022A80914405909145050E94300C2F
:102040006BEA75E080EE95E00E94442A68E875E04E
:1020500080EE95E00E94442A60E775E080EE95E00E
:102060000E94442A6BE475E080EE95E00E94442AC9
:1020700080EE95E00E94302A0E94C80E68C01216B9
:102080000CF065C0332727FD30958091460590E020
:10209000821793070CF45BC066E375E080EE95E071
:1020A0000E94022A60914305772767FD70954AE0F8
:1020B00050E080EE95E00E94F52A6BE075E080EE3E
:1020C00095E00E94022A10E008E280914705181767
:1020D000D0F5C12FD0E0CC0FDD1FC85BDA4F2881CF
:1020E00030E080914305992787FD90950197281747
:1020F000390739F56BEB71E080EE95E00E94252AF7
:102100004AE050E0602F80EE95E00E941C2B6FEBC0
:1021100071E080EE95E00E94252AE981EF70F0E001
:10212000EE0FFF1FEE56FC4F6081718180EE95E04F
:102130000E94252A63EC71E080EE95E00E94252A3A
:102140000F5F1F5FC2CF80EE95E00E94302ADF91C3
:10215000CF911F910F910895FF920F931F93CF93EB
:10216000DF93C3E8D5E0F12C8E0188818823D1F17B
:1021700065EC71E080EE95E00E94252A4AE050E08F
:102180006F2D80EE95E00E941C2B62ED71E080EED9
:1021900095E00E94252A2196F801208130E0A0E1F7
:1021A000B7E20E947C2D9B01AC01A0918205B0E0BA
:1021B0000E948B2DAB01BC018091790590917A052D
:1021C000A0917B05B0917C05480F591F6A1F7B1FAA
:1021D0002AE030E080EE95E00E942B2BF394F8E1AA
:1021E000FF12C2CFCDB7DEB7E5E00C942C2E1092D3
:1021F000DD0485E6EEEDF4E0DF011D928A95E9F756
:102200000895CF93C82F8F3719F0883009F045C053
:10221000E091DD04EE23D9F1E150E093DD04F0E03C
:10222000E252FB4F10826DE070E080EE95E00E947C
:102230005906C0E08091DD04C81760F4EC2FF0E08F
:10224000E252FB4F608170E080EE95E00E945906FB
:10225000CF5FF0CF60E270E080EE95E00E9459061B
:102260006DE070E080EE95E00E945906C0E080913C
:10227000DD04C81778F5EC2FF0E0E252FB4F6081E7
:1022800070E080EE95E00E945906CF5FF0CF67E0E6
:1022900080EE95E00E94282A1DC08B3119F40E941F
:1022A000F7101AC08D30C1F08A30B1F08091DD0492
:1022B000843668F76C2F70E080EE95E00E94590636
:1022C000E091DD0481E08E0F8093DD04F0E0E252C6
:1022D000FB4FC08380E001C081E0CF910895CF9390
:1022E000C82F0E946A286093C6047093C704809325
:1022F000C8049093C904C093DB04CC2329F040E0C8
:1023000051EE60E070E004C040E855E260E070E04B
:1023100080EE95E00E94B22CCF9108959091CA046E
:10232000492F4F7050E0BA016F5F7F4F292F30E087
:10233000E4E035952795EA95E1F76217730759F0C0
:10234000FA01E553FB4F808381E0890F8F70907F06
:10235000892B8093CA0408956EE770E080EE95E0C3
:102360000E9459060895A3E1B1E0E9EBF1E10C9474
:10237000062EE3E8F5E0712C8191882321F0739417
:1023800028E17212F9CF66ED71E080EE95E00E94CF
:10239000562A4AE050E0672D80EE95E00E94532BCC
:1023A00080E00E947E0A0E94590B8E010E5F1F4F33
:1023B000C12CD12C7601C39466246A945C2C0E94B3
:1023C0005E284B015C012091820530E0A0E1B7E27C
:1023D0000E947C2D9B01AC01C701B6010E949E2D7D
:1023E0002091790530917A0540917B0550917C05CB
:1023F000620F731F841F951F2091B9053091BA0594
:102400004091BB055091BC0526173707480759076F
:1024100018F4F801608225C08C2D0E94B20961E099
:1024200070E080E090E00E948D28F80110820E9408
:102430005E28681979098A099B09643F7140810502
:10244000910540F40E94C809F8019081981778F727
:102450008083EDCF50FE03C02C982D9A02C02C9A99
:102460002D982FEFC21AD20AE20AF20A0F5F1F4F0D
:102470008FEFC816D104E104F10409F09FCFCE011B
:102480009395FC01D82E7FEF68EC2E2F281B271583
:1024900010F051E056C0DE01129651E02FEF41E0FE
:1024A0003D91321710F0322F01C0452F5F5F5F3F23
:1024B00011F0232FF5CF4193242F30E0A1E0B0E0BD
:1024C000AC0FBD1FA20FB31F5C93413079F0DE014A
:1024D000A20FB31F5C93423049F0AFEFBFEFAC0FD8
:1024E000BD1FA20FB31F6C934E3F78F6A2E0B0E081
:1024F000AC0FBD1FA20FB31F7C934D3F30F6A3E07E
:10250000B0E0AC0FBD1FA20FB31F6C93BECF452F21
:10251000242F30E0FC01E20FF31F6081AFEFB0E049
:10252000AC0FBD1FA20FB31F2C91621748F441508E
:10253000DC01A40FB11D2C9120836C934111E8CFD5
:102540005F5F571520F3372D369520E0231770F481
:10255000DC01A20FB11D4C91522F530FFC01E50F6E
:10256000F11D50815C9340832E5FF0CFF3E8EF2E96
:10257000F5E0FF2E8C01802F8D19871598F4F80156
:10258000C1908F014AE050E06C2D80EE95E00E94F2
:102590001C2B6CE280EE95E00E94282AF701C19284
:1025A0007F01E9CF80EE95E00E94302A81E0CD5E88
:1025B000DE4FEFE00C94222E1F920F920FB60F9277
:1025C00011240F931F932F933F934F935F936F9318
:1025D0007F938F939F93AF93BF93EF93FF9340911C
:1025E000BD055091BE056091BF057091C00589B1D0
:1025F0008A019B01007411272227332783FB882738
:1026000080F990E0A0E0B0E0081719072A073B071F
:1026100009F468C080918400909185001092850033
:10262000109284002091A70421115CC045FD02C0D6
:1026300096958795853C29E09207C0F180910A0123
:1026400090E0A0E0B0E00CE176956795579547954E
:102650000A95D1F7411551056105710521F441E055
:1026600050E060E070E0481759076A077B07D8F42C
:1026700080910A018F3FB9F040E080910A0148172C
:1026800080F4842F90E0880F991FFC01E957FB4FDD
:1026900020813181FC01E55FFE4F318320834F5F54
:1026A000ECCF1092A80410920A011CC08D3B22E0CE
:1026B0009207A8F020910A01203188F410910A01B4
:1026C00021E0210F20930A010E94DE08E12FF0E0B3
:1026D000EE0FFF1FE957FB4F9183808303C08FEFFD
:1026E00080930A01FF91EF91BF91AF919F918F91DC
:1026F0007F916F915F914F913F912F911F910F911A
:102700000F900FBE0F901F90189583E0809380006C
:102710008AE1809381008FEF9FEF909389008093EF
:10272000880010926F0088E080936D00E8E6F0E08A
:1027300080818460808308950E94200D8091D2055D
:10274000843011F41092D20508956F3018F08695F8
:102750008058089589E0689F802D11240895A0E095
:10276000B0E0E5EBF3E10C940D2EC82F0E946A282F
:10277000009138041091390420913A0430913B04BF
:102780006B017C01C01AD10AE20AF30A97018601A3
:1027900049E8C41643E1D406E104F10410F01092B4
:1027A0003C04609338047093390480933A04909306
:1027B0003B042091A7048FEF820F8230D8F5E0917F
:1027C0003C04EE2309F44EC1E13011F482E0B8C1BB
:1027D000E03108F034C181E08E0F80933C04F0E0DA
:1027E000E957FB4FC083803109F0ACC1E9E8F4E060
:1027F000213029F4A181A695A695808108C0808109
:102800009181A92FA695A695A69596958795A03115
:1028100048F4B0E090E0AA0FBB1FA55FBE4F119631
:102820009C938E931092A804329684E0E739F807BF
:10283000F9F688C1233009F005C1E0913C04E111AB
:1028400004C0CF3009F07EC10DC1E83148F481E009
:102850008E0F80933C04F0E0EA57FB4FC08372C1B7
:10286000E83109F0ECC0C111EAC040E050E0ABE053
:10287000CA01B3E0880F991FBA95E1F7A49F9001B0
:10288000A59F300D1124F901E957FB4F6081E181CB
:102890007E2F777075956795FC01EE0FFF1FE55F42
:1028A000FE4F71836083F901E857FB4FB081B69505
:1028B000B695B695E181FE2FF295FF0FF07E6F2F52
:1028C0006B2BE695E695E6957E2F77707595679567
:1028D000FC01EE0FFF1FE35FFE4F71836083F90180
:1028E000E757FB4FB081B295B695B695B370C181ED
:1028F000DC2FDD0FDD0F6D2F6B2BC295C695C695B6
:10290000C370E281E170EE0FEE0F7E2F7C2B759588
:102910006795FC01EE0FFF1FE15FFE4F718360833F
:10292000F901E557FB4FB081B695E181FE2FF79590
:10293000FF27F7956F2F6B2BE6957E2F7770759598
:102940006795FC01EE0FFF1FEF5EFE4F7183608302
:10295000F901E457FB4FB081B295BF70E181FE2FC2
:10296000F295F07F6F2F6B2BE295EF707E2F7770D3
:1029700075956795FC01EE0FFF1FED5EFE4F7183AD
:102980006083F901E357FB4FB081BB1FBB27BB1F1F
:10299000C181DC2FDD0F6D2F6B2BCC1FCC27CC1F03
:1029A000E281E370EE0F7E2F7C2B75956795FC011D
:1029B000EE0FFF1FEB5EFE4F71836083F901E1575D
:1029C000FB4FB081B695B695E181FE2FF295FF0FD2
:1029D000FF0FF07C6F2F6B2BE695E6957E2F7770BF
:1029E00075956795FC01EE0FFF1FE95EFE4F718341
:1029F0006083F901E057FB4F2081229526952770CF
:102A00003181E32FEE0FEE0FEE0F6E2F622B732F3F
:102A100072957695777075956795FC01EE0FFF1F9F
:102A2000E75EFE4F718360834F5F5F4F4230510519
:102A300009F01ECF80919D0483FF1092A80410928C
:102A40003C0480C0243009F07DC060913C046111D9
:102A50000BC0C83AB1F4109273051092720588EA5F
:102A60000E94610681E06CC0613019F4C0933704A4
:102A700004C0623031F4C09336048C2F0E9461068A
:102A80005AC0E09136042E2F30E0220F331F462F1C
:102A900050E0C9010296841795073CF0633268F74D
:102AA000FA01EC57FB4FC083E8CF2D5F3F4F8C2FCF
:102AB00090E060917205709173054217530749F4D5
:102AC000982F882786279727909373058093720500
:102AD00032C06817790769F580913704813049F56C
:102AE000E13118F080E180933604F0903604C8E8B4
:102AF000D4E000E010E00F15D0F4FE0131978081A2
:102B000090E0982F88272881822B43E0969587951F
:102B10004A95E1F70E94DE08F801EE0FFF1FE55F1E
:102B2000FE4F918380830F5F1F4F2296E4CF109258
:102B3000A80410923C0480913C04882319F08F5F14
:102B400080933C04CDB7DEB7E8E00C94292EE82F43
:102B5000F0E0E854FA4FE185E03150F4F894F0E009
:102B6000EE0FFF1FE55FFE4F8081918178940895FD
:102B7000E03121F0E13131F483E101C082E10E94D2
:102B8000AC29089580E092E00895A2E2B0E0EBEC79
:102B9000F5E10C94032E9E012F5F3F4F80E1D90198
:102BA0001D928A95E9F764E072E080EE95E029A332
:102BB0003AA30E94562A0E947C0B1D8A1E8A1F8AF5
:102BC000188E312C212C00E0812C912C5401412CA9
:102BD00074E7572E7BE8672E72E3772EE0E5CE2E62
:102BE000E3ECDE2EE12CF12C84EF91E0A0E0B0E0EC
:102BF0008D8F9E8FAF8FB8A380E09EECADEEB4E3D7
:102C0000898F9A8FAB8FBC8F80E094E7ABE8B2E3FB
:102C1000898B9A8BAB8BBC8B80EE95E00E946A2BE4
:102C2000892B09F4E1C080EE95E00E94972B9C016E
:102C300033272C32310509F442C0ACF4233231057C
:102C400009F0ABC019821A821B821C821D821E826F
:102C50001F82188619861A861B861C861D861E866C
:102C60001F86188A60C02434310529F023353105C8
:102C700009F4B2C092C064E480EE95E00E94282A74
:102C80002AE030E040E054E76BE872E380EE95E044
:102C90000E94B62A6CE280EE95E00E94282A2AE083
:102CA00030E040E05EEC6DEE74E380EE95E00E9473
:102CB000B62A6CE280EE95E00E94682AADCF0F5FE5
:102CC000043009F0A9CF29813A814B815C81A8EEBB
:102CD000B3E00E948B2D698B7A8B8B8B9C8B2D8123
:102CE0003E814F8158850E948B2D698F7A8F8B8F03
:102CF0009C8F29853A854B855C852D8F3E8F4F8F24
:102D000058A32D853E854F8558890E948B2D6B01D8
:102D10007C0160323EE473078105910530F462E383
:102D20008CE10E949F0900E077CF603345E774078C
:102D30008105910510F462E2F3CF60345CE9750718
:102D40008105910510F466E2EBCF80E5C81683ECAF
:102D5000D806E104F10410F462E1E2CF90E6C9166E
:102D60009AEED906E104F10410F465E1D9CFA0E7A9
:102D7000CA16A1E1DA06A1E0EA06F10410F461E066
:102D8000CFCFB0EACB16B6E8DB06B1E0EB06F10434
:102D900010F463E0C5CF65E0C3CF10ED180F1A3013
:102DA00008F03ACFE1E0F0E0EC0FFD1F24E0029FD5
:102DB000E00DF11D11242081318142815381AAE06F
:102DC000B0E00E948B2D610F711D811D911D6083EC
:102DD00071838283938320CF49885A886B887C884B
:102DE000812C912C540118CF81149104A104B104B9
:102DF00089F4C301B2010E940E0A61E070E080E034
:102E000090E00E948D281D8A1E8A1F8A188E312C00
:102E100022242A948D8D9E8DAF8DB8A18816990697
:102E2000AA06BB06D0F40E94C8092D893E894F89A5
:102E3000588D280F311D411D511D2D8B3E8B4F8B01
:102E4000588F381608F4382E821508F4282E3FEFD4
:102E5000831A930AA30AB30A56C0C301B20128EE2B
:102E600033E040E050E00E94C22DBA01A9012AE0FF
:102E700030E080EE95E00E940D2B6CE280EE95E054
:102E80000E94282A4AE050E0632D80EE95E00E94DF
:102E90001C2B6CE280EE95E00E94282A6D897E89C9
:102EA0008F89988DA50194010E94C22DBA01A901B4
:102EB0002AE030E080EE95E00E940D2B6CE280EE7F
:102EC00095E00E94282A4AE050E0622D80EE95E0CD
:102ED0000E941C2B6CE280EE95E00E94682A4C0C4C
:102EE0005D1C6E1C7F1C898D9A8DAB8DBC8D8415ED
:102EF0009505A605B70520F449885A886B887C8813
:102F0000812C912C540129893A894B895C89283E6E
:102F100033404105510509F07FCEA296E2E10C94C1
:102F20001F2EACE1B0E0E7E9F7E10C940D2E0E9412
:102F30006A286B017C0181E00E947E0A14E703E0AD
:102F4000198361E0CE0101960E94DB0B00937105AD
:102F50000E94590B6AEF70E080E090E00E948D289B
:102F600080917105833089F480EE95E00E946A2B90
:102F7000892B59F40E946A286C197D098E099F09D2
:102F80006038734C894C9140D8F280917105833040
:102F900009F44FC08FE70E9477090E948A0989834C
:102FA000843511F083E05CC00E948A0910924405C8
:102FB000809345050E948A0920914405309145057A
:102FC000280F311D30934505209344050E948A093E
:102FD000809346050E948A0980934705813110F746
:102FE000F12C0F2D10E08091470590E0880F991F7C
:102FF0000817190740F40E948A09F801E85BFA4FA4
:103000008083F394EECF80E7898361E0CE0101965F
:103010000E94DB0B83E0809371050E94590B62E3F1
:1030200070E080E090E00E948D28809171058330EF
:1030300011F482E015C08FE70E9477090E948A0987
:103040008983803509F0AECF0DE915E00E948A0929
:10305000F80181938F01F5E0083B1F07B9F781E084
:103060006C96E8E00C94292E80914305992787FD02
:103070009095A92FB92FFC013196EB30F10508F09E
:1030800066C0EC5CFF4F0C943A2E62E778E080EE6D
:1030900095E00E94442A80E893E00E94300C6AE5A3
:1030A00078E080EE95E00E94442A65E378E080EEC7
:1030B00095E00E94442A6BE078E080EE95E00E9463
:1030C000442A6AEE77E080EE95E00E94442A6DEB98
:1030D00077E080EE95E00E94442A67E977E080EE91
:1030E00095E00E94442A63E777E080EE95E00E9435
:1030F000442A6CE477E080EE95E00E94442A80EE5A
:1031000095E00E94302A0E94610D21C06FE277E0B5
:103110001AC06AE077E017C065EF76E014C066ED8C
:1031200076E011C062E976E00EC06DE776E00BC094
:1031300068E676E080EE95E00E94442A62E276E05E
:1031400002C06CE076E080EE95E00E94442A6AE0DE
:1031500070E080E090E00E948D2880EE95E00E9473
:103160006A2B892B29F080EE95E00E94972BF5CFF2
:103170000895ACE1B0E0EFEBF8E10C940D2E9091E6
:1031800043059F3F09F023C1482F50E0FA013A97C9
:10319000EF36F10508F00FC1E15CFF4F0C943A2EB9
:1031A00061E172E0A0C06DE172E080EE95E00E9406
:1031B000562A85E789838BE1EDE9F5E0DE01129679
:1031C00001900D928A95E1F76CE1CE0101960E9483
:1031D000DB0B0E94590B83E08093710568EC70E073
:1031E00080E090E00E948D2880917105843009F084
:1031F000E2C08FE70E9477090E948A09898385359A
:1032000009F0D9C06DEE74E080EE95E00E94442A8A
:103210006FEC74E080EE95E00E94442A61EB74E06C
:1032200096C065E372E080EE95E00E94562A89E63A
:10323000898361E0CE0101960E94DB0B0E94590B4D
:1032400083E08093710568EC70E080E090E00E947C
:103250008D2880917105843009F0ADC08FE70E9400
:1032600077090E948A0989838E010E5F1F4F7E01B4
:103270004DE1E40EF11C0E948A09F80181938F014F
:10328000EE15FF05C1F78BE1FE013296ADE9B5E021
:1032900001900D928A95E1F78981893409F08BC0FC
:1032A00063E974E080EE95E00E94442A65E774E0EB
:1032B00080EE95E00E94442A67E574E048C06FE420
:1032C00072E080EE95E00E94562A8EEF80934305CF
:1032D00072C080528750805390914605981708F02D
:1032E00066C06EE572E080EE95E00E94562A63C0EB
:1032F00084E18093430560E274E029C085E1809316
:10330000430569EE73E023C086E18093430562EBD9
:1033100073E01DC087E18093430568E673E017C042
:1033200088E18093430567E573E011C089E18093EC
:10333000430563E473E00BC08AE1809343056EE2CA
:1033400073E005C08BE18093430566E073E080EE97
:1033500095E00E94442A2FC06CEE72E080EE95E06A
:103360000E94442A8091AB0591E01DC066ED72E099
:1033700080EE95E00E94442A8091AB0592E013C054
:1033800061EC72E080EE95E00E94442A8091AB05EA
:1033900094E009C066EA72E080EE95E00E94442A5B
:1033A0008091AB0598E089278093AB058FEF8093E0
:1033B00043050E94021080EE95E00E946A2B892B43
:1033C00009F45AC180EE95E00E94972BF4CF0E9439
:1033D0000111882309F450C18091DD04811104C0DA
:1033E0008FEF8093430540C140E050E060E070E023
:1033F0008EED94E00E94B12E40914305042F1127D9
:1034000007FD1095212F312FF8013197EB31F10590
:1034100008F01AC1E255FF4F0C943A2E552747FD8C
:1034200050952091460530E0241735070CF40CC167
:103430008B019C010150110921093109003211054C
:103440002105310558F0C0904705E9E4F5E0F12C7D
:10345000D12CA8E2EA2E415051090FC0FA01E356DF
:10346000FA4F61506083D8C0DF0111972C9130E092
:103470002417350729F0F3943296FC10F5CFCAC013
:103480000E2D10E020E030E0061717072807390757
:1034900041F42081DA01A356BA4F11962C93DD2412
:1034A000D394E394E8CF6F3F71058105910511F046
:1034B00008F0CAC06093B505AFC06F3F71058105C4
:1034C000910511F008F0C0C06093B605A5C06F3F2C
:1034D00071058105910511F008F0B6C06093B7053C
:1034E0009BC02091DE0420622037E9F440E050E0E8
:1034F00060E070E08FED94E00E94B12E9B01AC0182
:10350000DC01CB010197A109B1090897A105B1051B
:1035100008F0ADC0A4EDB0E30E948B2D6A5E7C4A3A
:103520008A46954E24C02636E9F440E050E060E03B
:1035300070E08FED94E00E94B12E9B01AC01DC01A4
:10354000CB010197A109B1090797A105B10508F0C1
:103550008EC0A8EAB1E60E948B2D645E7C438E4645
:10356000944E05C0611571058105910571F08B01BF
:103570009C0114572B4832430130FAE51F07F2E64D
:103580002F07F2E03F0708F05FC06093AD0570932E
:10359000AE058093AF059093B0053EC06F3F7105B7
:1035A0008105910511F008F04FC06093B10534C05A
:1035B0008B019C0101501109210931090F3F1105AF
:1035C0002105310508F040C06093B20525C08B018C
:1035D0009C01045C1940210931090D344DE11407A7
:1035E0002105310528F47093B4056093B30514C028
:1035F000611571058105910521F48FEF8093AC056C
:103600000BC06134710581059105F0F46150609340
:10361000AC0502C0DD20C1F08091DC0481111AC02C
:1036200080917D0590917E05A0917F05B0918005E8
:103630000196A11DB11D80937D0590937E05A093F9
:103640007F05B093800506C060E772E080EE95E0EC
:103650000E94562A0E94F7108FEF809343056AE07C
:1036600080EE95E00E94682A0E94021005C061E089
:1036700070E080E090E07BCF6C96E8E00C94292E1F
:103680006AE572E080EE95E00E94442A62E472E00E
:1036900080EE95E00E94442A80EE95E00E946A2B1D
:1036A000892B31F080EE95E00E94972B0E94B9188B
:1036B0000E949117823029F0833051F46DE072E05E
:1036C00002C064E272E080EE95E00E94442A089510
:1036D0008FEF809343051092DC040E9402108091CA
:1036E00043058E3F69F080EE95E00E946A2B892B9E
:1036F000B1F380EE95E00E94972B0E94B918EFCFAE
:1037000008950F931F93109143051F3F09F0D2C0F6
:10371000893409F457C000F5883309F469C058F4B6
:10372000803309F477C008F061C08B3109F440C0E0
:103730008132B1F1B9C0813409F487C030F48933E2
:1037400009F466C0803461F1AFC0823409F48EC0E0
:10375000863409F448C0A8C0823609F487C078F4DA
:10376000883531F128F48235C1F18335E1F09CC010
:103770008A3509F494C0813609F467C095C0823750
:1037800061F128F4863679F18936E1F08DC0883709
:1037900079F08A3709F483C0833709F085C003C004
:1037A00061E172E015C00E94320D6EE872E004C063
:1037B0000E943B0D68EA72E080EE95E00E94562A76
:1037C0008EEF70C00E947A060E94BF0667EC72E01E
:1037D00080EE95E00E94562A67C081E00E94DF06D5
:1037E00060EE72E0F5CF0E94AC105EC080535AC00C
:1037F0006AEF71E080EE95E00E94442A90919C056A
:1038000088E0890F8871977E892B80939C051AC068
:1038100089E048C067EE71E080EE95E00E94442A9E
:103820008091BD059091BE05A091BF05B091C005E6
:1038300020E182278093BD059093BE05A093BF052C
:10384000B093C005109343052FC061ED71E080EE89
:1038500095E00E94442A8091BD059091BE05A091FB
:10386000BF05B091C00540E4842710C060EC71E052
:1038700080EE95E00E94442A8091BD059091BE059E
:10388000A091BF05B091C00520E282278093BD05BD
:103890009093BE05A093BF05B093C00502C00E94DF
:1038A000401B8FEF80934305809143058E3F09F0C5
:1038B000D4C0DDC00E940111882309F4D8C08091D2
:1038C000DD04811104C08FEF80934305C6C040E042
:1038D00050E060E070E08EED94E00E94B12E009127
:1038E0004305112707FD1095212F312FF80131973E
:1038F000E930F10508F0B4C0E753FF4F0C943A2EBD
:103900008B019C01015014472B4832430F3F19454E
:103910002246324008F0A4C06093790570937A057E
:1039200080937B0590937C0577C060937D057093B1
:103930007E0580937F059093800581E08093DC0471
:103940006BC0683071058105910508F089C06093EE
:10395000810562C08B019C010150110921093109C7
:103960000A3011052105310508F07AC060938205FF
:1039700053C061EB71E08EED94E00E94EB2F10E0FC
:10398000009799F00E94C52F009779F0183130F414
:10399000E12FF0E0EC58FA4F87871F5F61EB71E091
:1039A00080E090E00E94EB2FEBCF1831A8F5E12FDB
:1039B000F0E0EC58FA4F17861F5FF7CF65307105BE
:1039C0008105910508F04CC060939B0525C08B01D3
:1039D0009C01015011092109310906301105210509
:1039E0003105F0F520919C05287F262B20939C051E
:1039F00013C08B019C0101501109210931090115E6
:103A0000124C2140310560F5609375057093760581
:103A100080937705909378058091DC04811113C021
:103A200080917D0590917E05A0917F05B0918005E4
:103A30000196A11DB11D80937D0590937E05A093F5
:103A40007F05B09380050E94F7108FEF80934305A8
:103A50006AE080EE95E00E94682A0E94341807C050
:103A600060E772E080EE95E00E94562AECCF1F914D
:103A70000F9108958FEF809343051092DC040E940C
:103A80003418809143058E3F69F080EE95E00E94E6
:103A90006A2B892BB1F380EE95E00E94972B0E9450
:103AA000811BEFCF6AE070E080E090E00E948D28FB
:103AB00080EE95E00E946A2B892B29F080EE95E03C
:103AC0000E94972BF5CF0895CF93C82F682F80EED3
:103AD00095E00E94C42B909168059C2790936805FF
:103AE000CF910895A1E0B0E0E8E7FDE10C94132E3A
:103AF00099830E94641D9981892F0E94641D2196DB
:103B0000E2E00C942F2E1F93CF93DF93182FEB013D
:103B10001092680565EB70E080EE95E00E94590612
:103B200062E670E080EE95E00E945906812F0E94C7
:103B3000641DCE010E94721DDF91CF911F910895E7
:103B40006091680580EE95E00E94C42B0895A1E283
:103B5000B0E0EDEAFDE10C940F2E7B018A018C3080
:103B600009F453C108F040C0863009F4BCC018F510
:103B7000833009F491C070F4813009F472C082304E
:103B800009F048C26BE170E082E00E94831D0DE9FC
:103B900015E078C0843009F487C0853009F03AC256
:103BA0006091470570E0660F771F85E00E94831DD6
:103BB00008E415E086C0893009F4A7C070F48730A6
:103BC00009F49BC0883009F025C261E070E088E00C
:103BD0000E94831D8091D20523C28A3009F4CAC095
:103BE0008B3009F4F2C016C28A3609F475C1D8F4D4
:103BF000873609F43AC138F4853609F40EC18636A1
:103C000009F41FC107C2883609F437C1893609F0A3
:103C100001C261E070E089E60E94831D0E947A067D
:103C20000E94BF06F5C18D3609F4D4C138F48B3635
:103C300009F491C18C3609F49AC1ECC18E3609F4AD
:103C4000DCC1873C09F0E6C161E070E087EC0E94CE
:103C5000831D81E00E94641D0E94A01D10926905D1
:103C6000E3C169E270E081E00E94831D04E715E092
:103C7000F80181918F010E94641DF5E00D391F0745
:103C8000B9F7D0C1F80181918F010E94641DF5E060
:103C9000083B1F07B9F7C6C161E070E083E00E94EE
:103CA000831D0E949117BCC161E070E084E00E9416
:103CB000831D81E00E94641D0E94A01D0E94C51505
:103CC000B3C18091470590E0880F991F980128544F
:103CD00035402817390708F0A5C1F80181918F01F7
:103CE0000E94641DEECF62E070E086E00E94831DBA
:103CF00080E893E00E94721D95C161E070E087E06A
:103D00000E94831D809146058BC186E6898361E010
:103D1000CE0101960E94DB0B0E94590B83E0809339
:103D2000710568EC70E080E090E00E948D28809141
:103D300071058430D9F48FE70E9477090E948A09BF
:103D40008983863469F460E270E089E00E94831D13
:103D500010E20E948A090E94641D1150D1F762C1CD
:103D600061E070E089E00E94831D52C161E070E073
:103D700089E053C169E170E08AE00E94831D81E01F
:103D80008093B805209170058091BD059091BE0586
:103D9000A091BF05B091C005222311F0806801C039
:103DA0008F778093BD059093BE05A093BF05B09318
:103DB000C00508EB15E0F80181918F010E94641D98
:103DC000F5E0013D1F07B9F72DC161E270E08BE01E
:103DD0000E94831D8091A8048F3F39F08091A80430
:103DE00091E0980F9093A80402C08091A8040E94CB
:103DF000641D10E0812F0E94A7150E9409090E94EE
:103E0000721D1F5F1031B1F70DC161E070E08CE0F1
:103E10000E94831D8091D10503C161E070E085E6B9
:103E20000E94831D89E2E816F10409F0F8C0D80168
:103E3000E4E7F5E08D91819385E0ED39F807D1F75E
:103E4000E7C061E070E086E60E94831DEBE1EE16BC
:103E5000F10409F0E4C0D801EDE9F5E08D9181931A
:103E600085E0E83BF807D1F7D3C061E070E087E672
:103E70000E94831D0E94320DCBC061E070E088E695
:103E80000E94831D85E789838BE1EDE9F5E0DE0182
:103E9000129601900D928A95E1F76CE1CE010196A0
:103EA0000E94DB0B0E94590B83E08093710560E256
:103EB00073E080E090E00E948D288091710584304D
:103EC00009F0ADC08FE70E9477090E948A098983B3
:103ED000853509F0A4C09CC061E070E08AE60E94CC
:103EE000831D89E6898361E0CE0101960E94DB0B88
:103EF0000E94590B83E08093710560E273E080E0DB
:103F000090E00E948D2880917105843009F087C06F
:103F10008FE70E9477090E948A0989838E010E5FCC
:103F20001F4F7E01EDE1EE0EF11C0E948A09F8019F
:103F300081938F01EE15FF05C1F78BE1FE013296EB
:103F4000ADE9B5E001900D928A95E1F78981893458
:103F500009F065C05DC061E070E08BE60E94831DE2
:103F6000F80180818093D2050E943B0D51C061E031
:103F700070E08CE60E94831DF0E2EF16F10461F41C
:103F800087E6898380E2F801DE01129601900D92A6
:103F90008A95E1F761E203C087E4898361E0CE019D
:103FA00001960E94DB0B0E94590B83E08093710500
:103FB0006CE474E080E090E00E948D2880917105AF
:103FC000843069F58FE70E9477090E948A09873457
:103FD00031F51EC061E070E08DE60E94831D89E12D
:103FE000E816F104E1F4D801E8EBF5E08D91819356
:103FF00085E0E13DF807D1F70BC061E070E08EE6A7
:104000000E94831DF80180818093D1050E941B0DC1
:1040100081E006C061E070E08AEC0E94831D80E0D0
:104020000E94641D0E94A01DA196E6E00C942B2E18
:10403000A0E0B0E0EEE1F0E20C940D2ECAECD3E08B
:1040400014E606E035E0F32E44E0E42E53E0D52EEE
:1040500062E0C62E80EE95E00E946A2B892B09F45F
:104060009BC080EE95E00E94972B282F809335040B
:104070004091340450E04730510560F7FA01EE52A8
:10408000FF4F0C943A2E853B29F781E0809334044E
:10409000E1CF823609F07DC0C0923404DBCF80933B
:1040A000330480933204D0923404D4CF9C0133275C
:1040B00030933104209330049091320498279093E8
:1040C0003204E0923404C6CF382F222740913004C6
:1040D00050913104242B352B30933104209330043C
:1040E00090913204982790933204F092340425364C
:1040F000310508F4AFCF61E070E08CEC0E94831DC5
:1041000081E00E94641D0E94A01D43C020912E04E6
:1041100030912F04F901E653FC4F808390913204D3
:10412000982790933204C901019690932F048093AD
:104130002E0420913004309131048217930708F443
:1041400089CF0093340486CF8091320482130BC050
:1041500060912E0470912F044AEC53E08091330457
:104160000E94A71D0DC062E070E08BEC0E94831DD1
:10417000809133040E94641D809168050E94641D33
:10418000FE01812F11928A95E9F710922F04109267
:104190002E04109234045ECFCDB7DEB7E8E00C9465
:1041A000292E81E08093690580916905882349F073
:1041B00080EE95E00E946A2B892BB1F30E941820B3
:1041C000F3CF0895AAE2B0E0E8EEF0E20C940B2EF3
:1041D0000E945E286B017C0181E00E947E0A80EED5
:1041E00095E00E946A2B892B29F080EE95E00E94D1
:1041F000972BF5CF2D9811E072E6B72EE9E2AE2E9F
:1042000003E00E945E286C197D098E099F09693CB4
:10421000710581059105D0F11123C1F10E945E283D
:104220006B017C012C9A80ED97E00E94A807B9826F
:10423000E4E7F5E0DE0112968A2D01900D928A9551
:10424000E1F76AE2CE0101960E94DB0B2C9880E038
:1042500090E00E94A807009371050E94590B62E349
:1042600070E080E090E00E948D288091710584309C
:1042700061F4009371058FE70E9477090E948A0913
:1042800011E0823419F410E001C011E08BE00E94CB
:104290008329892B81F411E00EC02D9A2C9A80EE8F
:1042A00095E00E94972B8D309105A9F05CF40A9758
:1042B00091F02D982C9880EE95E00E946A2B892B26
:1042C00061F79FCF8332910579F08234910589F7A8
:1042D0000E94D120EECF62EB71E080EE95E00E946B
:1042E000442A0E943A1DE5CF0E94C515E2CF8F9265
:1042F0009F92AF92BF92CF92DF92EF92FF921F9365
:10430000CF93DF938BE00E948329892B09F089C02A
:1043100068EC70E080E090E00E948D2880E090E002
:104320000E94A8070E945E284B015C016B017C0182
:1043300080ECC80E82E1D81EE11CF11C0E945E28B0
:104340006C157D058E059F0530F48BE00E94832956
:10435000892BA1F364C08BE00E948329892B09F08B
:104360005EC080ED97E00E94A8070E945E286B0166
:104370007C01D0E0C1E088E4880E86E2981EA11C92
:10438000B11C11E08BE00E948329892B21F58C144C
:104390009D04AE04BF0430F480ED97E00E94A807AE
:1043A000D1E0F0CF0E945E286C197D098E099F092B
:1043B000693C71058105910528F30E945E286B0117
:1043C0007C01C12719F080ED97E002C080E090E009
:1043D0000E94A807D7CF80E090E00E94A807DD23C5
:1043E000B9F08091D10590E0019665E070E00E94FF
:1043F000AE2D8093D1050E941B0D0E949C130E943C
:104400003B0D64EF71E080E090E00E948D2809C0D0
:1044100080E00E94DF060E94B3110E94320D0E94CC
:10442000E220DF91CF911F91FF90EF90DF90CF902E
:10443000BF90AF909F908F900895CF92DF92EF92B0
:10444000FF9280E00E94DA070E94B10761E08DE0F0
:104450000E94172961E08CE00E94172960E08BE040
:104460000E94172960E083E00E94172961E083E041
:104470000E94502961E08EE00E94172960E08EE0E2
:104480000E9450290E949F0740E052EC61E070E0DA
:1044900080EE95E00E94B22C0E949C130E943B0D7E
:1044A0000E9485138FEF8093A8040E94C60778941A
:1044B0000E945E286B017C018091A8048F3F59F413
:1044C0000E945E286C197D098E099F09603D774026
:1044D0008105910588F380ED97E00E94A80761E0CF
:1044E0008BE00E9450292D9A80EE95E00E946A2B65
:1044F000892B29F080EE95E00E94972BF5CF6DEF88
:1045000072E080EE95E00E94252A80E893E00E9408
:10451000300C64E173E080EE95E00E94252A4AE0C9
:1045200050E062E070E080EE95E00E94F52A62E3E0
:1045300070E080E090E00E948D2880EE95E00E947F
:104540006A2B04970CF180EE95E00E94972B823441
:104550009105D1F480EE95E00E94972B8E34910561
:1045600099F480EE95E00E94972B8434910561F4D4
:1045700080EE95E00E94972B819731F480E090E0E7
:104580000E94A8070E94E22040917505509176058F
:104590006091770570917805DB01CA010197A10947
:1045A000B1090497A105B10568F44093A70443300D
:1045B00029F440EA56E861E070E004C040E052ECC3
:1045C00061E070E080EE95E00E94B22C0E947721BD
:1045D0002D9880E090E00E94A8070E948513109219
:1045E000C3048091BD0583FF11C080918905882394
:1045F00051F080919005882331F0809197058823B0
:1046000011F087E001C085E08093C30480E00E9440
:104610007E0A8091C4040E94B2090E94590B109234
:104620003F0410923E0410923D04F12C8091D2057B
:104630008F15B0F062E370E080E090E00E948D287A
:1046400080ED97E00E94A80762E370E080E090E0D0
:104650000E948D2880E090E00E94A807F394E6CFA6
:1046600080919C0584FF08C0982F987181E0983153
:1046700009F080E00E946F118FE00E94DA07FF903E
:10468000EF90DF90CF900895EF92FF920F931F93DA
:10469000CF93DF938C016EE770E080EE95E00E948F
:1046A0005906E801F12CF0E2EF2E8E0188818D573A
:1046B000823048F46DE770E080EE95E00E94590684
:1046C00088818E2588832196F801608180EE95E0AF
:1046D0000E94C42BF394F9E0FF12E7CF6EE770E07D
:1046E00080EE95E00E945906CDB7DEB7E6E00C9467
:1046F0002B2EA9E0B0E0EFE7F3E20C94132E90919B
:10470000C50491110EC09EEF99838A836B8350E09C
:10471000559547954C832D83198618861F821E82D6
:104720002EC04091CA04842F90E0B4E095958795FF
:10473000BA95E1F7242F2F7030E08217930719F113
:104740008DEF89831B82FE01349650E0842F90E028
:10475000A4E095958795AA95E1F7242F2F7030E076
:104760008217930749F0DC01A553BB4F8C918193CD
:10477000405F5F5F563051F74093CA045A83CE01C1
:1047800001960E9444238091C50490E0019666E062
:1047900070E00E94AE2D8093C5042996E2E00C944F
:1047A0002F2EA0E0B0E0E7EDF3E20C940C2E6C01AC
:1047B0006EE770E080EE95E00E9459068601E12CDC
:1047C000F12CC0E0D0E030E2B32EF801608183E844
:1047D000860F823078F46DE770E080EE95E00E94FD
:1047E0005906F80160816B2570E080EE95E00E942B
:1047F000590604C080EE95E00E94C42BE114F10438
:1048000059F0F80180819E01280F311DC901C92F7F
:10481000DD27C80FD91FDD273FEFE31AF30A89E030
:10482000E816F10459F028E0E216F10421F48C2F87
:104830008095F60180870F5F1F4FC7CFCDB7DEB7DA
:10484000E9E00C94282EA9E0B0E0E9E2F4E20C944F
:10485000132EE82F362F8091C50490E0019664E274
:1048600070E00E94AE2D8093C50458E9598350E151
:104870005A83813089F048F08230B9F08330D9F41E
:104880008B8381EF8C833D8319C085E08B8381EF1F
:104890008C832F5F2D8312C08B8381EF8C8384E602
:1048A000489FA00111245D8309C084E08B8381EFC0
:1048B0008C83ED8303C00E94AC1104C0CE0101962D
:1048C0000E94D1232996E2E00C942F2EA2E0B0E0C2
:1048D000ECE6F4E20C94082E182F762E2A834983F6
:1048E0000E946A286B017C018091DB048090C604E1
:1048F0009090C704A090C804B090C9042A8149814F
:104900008823C1F0D701C60188199909AA09BB09F2
:104910004C015D0191EE89169EE29906A104B10455
:1049200020F1241708F4422F202F672D812F0E9499
:10493000232413C0D701C60188199909AA09BB0904
:104940004C015D0191E3891695E79906A104B10434
:1049500060F0672D812F0E947923C092C604D09207
:10496000C704E092C804F092C9042296EDE00C94CA
:10497000242EA2E2B0E0EFEBF4E20C94092E8CE0DE
:104980000E94990981110DC06CE173E080EE95E001
:104990000E94562A2D9A80E00E947E0A0E94590B9E
:1049A0002D9880EE95E00E946A2B892B01F180EE14
:1049B00095E00E94972B9091A704992319F00E94EB
:1049C000AF13EFCF40913E0450E09A012F5F3F4F6D
:1049D0002F71332760913F0470E02617370709F3E2
:1049E000FA01E75BFB4F808320933E04DACF80918E
:1049F0007105843009F086C00E946A28611571052E
:104A00008105910549F06093B5047093B6048093D5
:104A1000B7049093B8040CC081E090E0A0E0B0E04F
:104A20008093B5049093B604A093B704B093B804F0
:104A30008091AB049091AC0481609093AC0480931E
:104A4000AB0483E0809371058FE70E94770909E644
:104A500014E00E948A09F80181938F01F4E0023783
:104A60001F07B9F72091720480916904982F92274B
:104A700096FF3BC090E4922790937204982F98730E
:104A80009833F1F410E0212F30E0809169048770B1
:104A900090E0821793074CF11F5F20919C05812FB6
:104AA00090E0FC01E759FB4F24FF04C080810E9485
:104AB0008E11E9CF608180EE95E00E94C42BE3CF98
:104AC0008F7399F480916A048093B40480916B048D
:104AD0008093B20480916C048093B10480916F0440
:104AE00090E09093AA048093A90480913D048130C2
:104AF00019F482E080933D0480913D04833011F4E9
:104B000010923D040E946A286B017C018091AD04E3
:104B10009091AE04A091AF04B091B0040097A105AC
:104B2000B105C9F0A7019601281B390B4A0B5B0B95
:104B3000DA01C901883B9B40A105B10560F00E94E4
:104B4000C8098093B3041092AD041092AE04109281
:104B5000AF041092B0048091B9049091BA04A0916E
:104B6000BB04B091BC0446015701881A990AAA0AED
:104B7000BB0A84E795E00E94F40786169706A8060C
:104B8000B90608F4A8C0C092B904D092BA04E09261
:104B9000BB04F092BC040E9457068091A8048830A0
:104BA000A0F08091BD059091BE05A091BF05B09188
:104BB000C0056CE1B695A795979587956A95D1F74D
:104BC000892B8A2B8B2B09F0A4C18091A8048F5FBD
:104BD0008093A8048091B5049091B604A091B70485
:104BE000B091B8040097A105B105F1F0C81AD90A2F
:104BF000EA0AFB0A84E795E00E94F4076C157D053C
:104C00008E059F0508F006C18091BD0584FD04C096
:104C100080ED97E00E94A8071092B5041092B604A8
:104C20001092B7041092B80490917204907C909303
:104C3000720450913E0480913F0420913D04581726
:104C400009F405C1223009F002C190589093720412
:104C5000E0919C05E770F0E0E658FC4F6081693018
:104C600008F0DDC0615040E04613DBC080933F0494
:104C700087E3840F90917204892B80937204409390
:104C8000400483E080933D042C9A809181059091AB
:104C9000C30491112FC10E94790A8091C4040E941B
:104CA000B209E0919C05E770F0E0E658FC4F6081A6
:104CB00082E794E00E94940BE091C404EF5FE093DC
:104CC000C404E83109F422C1F0E0EC58FA4F8785BA
:104CD000882309F41BC10E94030C813069F580917F
:104CE0009C05887149F18091AB049091AC04880FC8
:104CF000991F9093AC048093AB0483E0809371057B
:104D00000E94590B0E946A286093AD047093AE0410
:104D10008093AF049093B004672B682B692B61F4E8
:104D200081E090E0A0E0B0E08093AD049093AE0409
:104D3000A093AF04B093B00480919C0584FF1FC082
:104D40008091AB049091AC048E7F0E942A09182FA9
:104D50006091A9048091B4040E94A513482F612F8B
:104D60008091B30449A30E94A5130091D205282F76
:104D700049A16091B1048091B2040E9466242C98EC
:104D80008091C1048130C1F018F08230B1F1CEC001
:104D90008BE00E948329892B09F0C8C081E08093B1
:104DA000C1040E945E286093BD047093BE0480938A
:104DB000BF049093C004BAC08BE00E948329892B62
:104DC00031F50E945E28C090BD04D090BE04E090F2
:104DD000BF04F090C0046C197D098E099F09693EDB
:104DE00073408105910508F4A1C082E08093C1045D
:104DF00080ED97E00E94A80799C08BE00E9483296C
:104E0000892B09F493C080E090E00E94A8071092DB
:104E1000C1048CC080E090E00E94A80705CF68E044
:104E200022CF851709F422CF4F5F242F30E090E086
:104E3000F901EE58FB4FDC01A75BBB4F7C917083FF
:104E4000F901E05CFB4F708301968F710DCF243028
:104E5000B1F42091400481E494E0A3E7B4E0FC01C4
:104E60003E2F381B321718F431913D93F9CF87E369
:104E7000820F90917204892B8093720402CF8091EB
:104E8000C104823069F49160909372042D9A51ECC0
:104E9000E52E55E0F52E8E010F5F1F4FB80110C0B3
:104EA0002D9880913D04811103C081E080933D04E1
:104EB00080913D04833059F784E080933D04E7CF2F
:104EC000F70181917F0169A37AA30E94A715F801D8
:104ED000819391938F0169A17AA1F1EDEF16F5E02D
:104EE000FF0671F780919C0543E754E087700E94AC
:104EF0007908CACE882309F4CECE2091C20431E0CD
:104F0000320F3093C2042913C6CE0CC01092C404D1
:104F1000E2CE8091A804883009F42D9A89E080932C
:104F2000A804D9CE1092C2048150B5CEA296ECE06E
:104F30000C94252E8230E8F4E82FF0E0EE0FFF1FEE
:104F4000ED52FA4F71836083813041F080916900A6
:104F50008C7F842B80936900E89A08958091690082
:104F6000440F551F440F551F837F842B8093690086
:104F7000E99A08951F920F920FB60F9211242F9362
:104F80003F934F935F936F937F938F939F93AF93D1
:104F9000BF93EF93FF938091D3059091D405892B14
:104FA00029F0E091D305F091D4050995FF91EF9197
:104FB000BF91AF919F918F917F916F915F914F9131
:104FC0003F912F910F900FBE0F901F9018951F9239
:104FD0000F920FB60F9211242F933F934F935F932D
:104FE0006F937F938F939F93AF93BF93EF93FF93B1
:104FF0008091D5059091D605892B29F0E091D505B2
:10500000F091D6050995FF91EF91BF91AF919F91D6
:105010008F917F916F915F914F913F912F910F9061
:105020000FBE0F901F9018951F920F920FB60F9200
:1050300011242F933F938F939F93AF93BF938091AE
:10504000D8059091D905A091DA05B091DB05309192
:10505000D70523E0230F2D3720F40196A11DB11DA4
:1050600005C026E8230F0296A11DB11D2093D70588
:105070008093D8059093D905A093DA05B093DB050A
:105080008091DC059091DD05A091DE05B091DF05F2
:105090000196A11DB11D8093DC059093DD05A093C1
:1050A000DE05B093DF05BF91AF919F918F913F9146
:1050B0002F910F900FBE0F901F9018952FB7F89457
:1050C0006091D8057091D9058091DA059091DB0542
:1050D0002FBF08953FB7F8948091DC059091DD05CE
:1050E000A091DE05B091DF0526B5A89B05C02F3F36
:1050F00019F00196A11DB11D3FBF6627782F892F9A
:105100009A2F620F711D811D911D42E0660F771F5E
:10511000881F991F4A95D1F70895CF92DF92EF9299
:10512000FF92CF93DF936B017C010E946A28EB0111
:10513000C114D104E104F10479F00E946A286C1BC7
:105140007D0B683E7340A0F381E0C81AD108E108E6
:10515000F108C851DC4FECCFDF91CF91FF90EF9079
:10516000DF90CF900895789484B5826084BD84B533
:10517000816084BD85B5826085BD85B5816085BD52
:10518000EEE6F0E0808181608083E1E8F0E010826B
:10519000808182608083808181608083E0E8F0E0AC
:1051A000808181608083E1EBF0E080818460808396
:1051B000E0EBF0E0808181608083EAE7F0E08081CD
:1051C000846080838081826080838081816080832D
:1051D0008081806880831092C1000895833081F0BF
:1051E00028F4813099F08230A1F008958630A9F03A
:1051F0008730B9F08430D1F4809180008F7D03C076
:10520000809180008F7780938000089584B58F7798
:1052100002C084B58F7D84BD08958091B0008F77E2
:1052200003C08091B0008F7D8093B0000895CF932C
:10523000DF9390E0FC01ED50F44F2491FC01E95F15
:10524000F34F8491882349F190E0880F991FFC0166
:10525000E15DF34FA591B4918B5D934FFC01C59136
:10526000D4919FB7611108C0F8948C912095822346
:105270008C93888182230AC0623051F4F8948C9117
:10528000322F309583238C938881822B888304C0AE
:10529000F8948C91822B8C939FBFDF91CF910895CE
:1052A000A1E0B0E0E6E5F9E20C94112E282F30E001
:1052B000F901E152F44F8491F901ED50F44F14914A
:1052C000F901E95FF34F04910023C9F0882321F02D
:1052D00069830E94EE286981E02FF0E0EE0FFF1F46
:1052E000EB5DF34FA591B4919FB7F8948C91611148
:1052F00003C01095812301C0812B8C939FBF219601
:10530000E4E00C942D2ECF93DF93282F30E0F901A9
:10531000E152F44F8491F901ED50F44FD491F90129
:10532000E95FF34FC491CC2391F081110E94EE28E4
:10533000EC2FF0E0EE0FFF1FE55EF34FA591B49167
:105340002C912D2381E090E021F480E002C080E0E8
:1053500090E0DF91CF9108958E3008F08E508770E5
:1053600020919D0190E4299F90011124822B80932C
:105370007C0080917A00806480937A0080917A002A
:1053800086FDFCCF809178002091790090E0922BEF
:105390000895A0E0B0E0EFECF9E20C940D2E6C0162
:1053A0007A01EB01E60EF71E00E010E0CE15DF05F6
:1053B00061F06991D601ED91FC910190F081E02DB1
:1053C000C6010995080F191FF1CFC801CDB7DEB787
:1053D000E8E00C94292E6115710589F0DB010D9030
:1053E0000020E9F7AD0141505109461B570BDC0184
:1053F000ED91FC910280F381E02D0995089580E004
:1054000090E00895EF92FF920F931F93CF93DF9355
:105410008C01FB01C0E0D0E064917F018FEFE81ABE
:10542000F80A662361F0D801ED91FC910190F081BA
:10543000E02DC8010995C80FD91FF701EDCFCE01A6
:10544000CDB7DEB7E6E00C942B2E0E94EB29089531
:10545000DC01ED91FC910190F081E02D099508951A
:105460000F931F93CF93DF93EC016DE00E94282AE6
:105470008C016AE0CE010E94282A800F911FDF91E3
:10548000CF911F910F9108950F931F93CF93DF93A7
:10549000EC010E94022A8C01CE010E94302A800F6A
:1054A000911FDF91CF911F910F9108950F931F933B
:1054B000CF93DF93EC010E94EB298C01CE010E9477
:1054C000302A800F911FDF91CF911F910F91089586
:1054D0000F931F93CF93DF93EC010E94282A8C0136
:1054E000CE010E94302A800F911FDF91CF911F9132
:1054F0000F910895A1E2B0E0E0E8FAE20C94092EE1
:105500007C01C42EE52FCB01D22E19A221E02D154E
:1055100010F02AE0D22E8E010F5D1F4F8D2C912CA2
:10552000A12CB12C6C2D7E2FA50194010E94C22DBF
:105530008C2DD29E80191124015011098A3010F44B
:10554000805D01C0895CF80180832115310541052A
:10555000510521F0C22EE32FCA01E4CFB801C701E3
:105560000E94EB29A196ECE00C94252EA0E0B0E07F
:10557000ECEBFAE20C940D2EEC016A017B01211593
:10558000310541F4E881F9810190F081E02D642F2B
:1055900009951DC02A303105A9F477FF12C06DE2CC
:1055A0000E94282A8C0144275527BA014C195D090D
:1055B0006E097F092AE0CE010E947A2A800F911F8E
:1055C00006C02AE0B701A601CE010E947A2ACDB713
:1055D000DEB7E8E00C94292E9A01AB01662757FD4F
:1055E0006095762F0E94B62A08950F931F93CF934C
:1055F000DF93EC019A01AB01662757FD6095762F8A
:105600000E94B62A8C01CE010E94302A800F911F81
:10561000DF91CF911F910F9108952115310549F424
:10562000DC01ED91FC910190F081E02D642F099552
:1056300008950E947A2A08959A01462F50E060E06A
:1056400070E00E940D2B08959A01AB0160E070E0BC
:105650000E940D2B08950F931F93CF93DF93EC01BE
:105660000E940D2B8C01CE010E94302A800F911FC9
:10567000DF91CF911F910F9108950F931F93CF93B7
:10568000DF93EC019A01AB0160E070E00E940D2B0A
:105690008C01CE010E94302A800F911FDF91CF91A3
:1056A0001F910F9108950F931F93CF93DF93EC01F8
:1056B0009A01462F50E060E070E00E940D2B8C01B3
:1056C000CE010E94302A800F911FDF91CF911F9150
:1056D0000F910895FC0124853585F901E05CFF4FA9
:1056E00080819181F901EE5BFF4F20813181821B26
:1056F000930B8F7399270895FC0184859585FC0190
:10570000E05CFF4F40815181FC01EE5BFF4F208147
:1057100031814217530741F00190F081E02DE80FED
:10572000F91F808190E008958FEF9FEF0895FC01AD
:1057300084859585FC01E05CFF4F40815181FC012F
:10574000EE5BFF4F208131814217530779F0A08132
:10575000B181A80FB91F8C91208131812F5F3F4FFC
:105760002F7333273183208390E008958FEF9FEFCD
:105770000895FC0181A1882329F0A489B5898C9121
:1057800086FFFBCF11A20895CF93DF93FC012685FE
:105790003785D901A05CBF4F8D919C9111970196DF
:1057A0008F739927E901CE5BDF4F488159818417B8
:1057B0009507D9F30D90BC91A02DA20FB31F6C9348
:1057C000A685B785A05CBF4F11969C938E93A68942
:1057D000B7892C9181E090E0078C02C0880F991F57
:1057E0000A94E2F7282B2C9381E081A30488F589A1
:1057F000E02D80818064808381E090E0DF91CF9113
:10580000089508951F920F920FB60F9211242F93AF
:105810003F934F938F939F93EF93FF938091C0009B
:1058200082FD1CC04091C60080918606909187063B
:1058300001968F73992720918806309189068217E7
:10584000930771F0E0918606F0918706EA5BF94FC5
:105850004083909387068093860602C08091C6009D
:10586000FF91EF919F918F914F913F912F910F90C9
:105870000FBE0F901F90189580EE95E00E946A2B46
:10588000892B11F00E94012C08951F920F920FB6E0
:105890000F9211242F933F938F939F93EF93FF9336
:1058A000209142063091430680914406909145062E
:1058B0002817390731F48091C1008F7D8093C10092
:1058C00014C0E0914406F0914506EE5FF94F208147
:1058D000809144069091450601968F739927909385
:1058E0004506809344062093C600FF91EF919F9157
:1058F0008F913F912F910F900FBE0F901F90189591
:10590000A0E0B0E0E6E8FCE20C94092EFC01138272
:10591000128288EE93E0A0E0B0E084839583A683B2
:10592000B7838CEB93E09183808375876487578777
:105930004687318B208B138B028BF58AE48AD78ABA
:10594000C68AB18EA08E938E828E8F85848F888931
:10595000858F8989868F8A89878F8B8980A3ECE0E0
:105960000C94252ECF92DF92EF92FF92CF93DF938C
:10597000EC016A017B01411581EE58076105710553
:10598000F9F0EC89FD8981E090E008A002C0880F61
:10599000991F0A94E2F7808360E079E08DE390E05C
:1059A000A70196010E94C22D2150310941095109D8
:1059B0005695479537952795211580E1380798F03A
:1059C000EC89FD89108260E874E88EE190E0A7011F
:1059D00096010E94C22D2150310941095109569565
:1059E000479537952795E889F9893083EA89FB89B6
:1059F000208319A2EE89FF89408181E090E09C011B
:105A00000C8C02C0220F331F0A94E2F7422B408312
:105A1000EE89FF8940819C010D8C02C0220F331F4B
:105A20000A94E2F7422B4083EE89FF8940819C0172
:105A30000E8C02C0220F331F0A94E2F7422B4083E0
:105A4000EE89FF8920810F8C02C0880F991F0A946C
:105A5000E2F7809582238083DF91CF91FF90EF90D2
:105A6000DF90CF9008958F929F92AF92BF92CF9286
:105A7000DF92EF92FF920F931F9381E08F9385E067
:105A80008F9387E08F9383E08F9384E08F93E6EC8E
:105A90008E2E912CF2ECAF2EB12CA1ECCA2ED12C73
:105AA000B0ECEB2EF12C04EC10E025EC30E042E001
:105AB00056E066E476E080EE95E00E94802C0F9040
:105AC0000F900F900F900F901F910F91FF90EF90FC
:105AD000DF90CF90BF90AF909F908F9008950E94DD
:105AE000B3280E941D22CCE3DCE20E94B924209757
:105AF000E1F30E943C2CF9CFA29FB001B39FC001FB
:105B0000A39F700D811D1124911DB29F700D811DE9
:105B10001124911D08950E947C2DA59F900DB49F86
:105B2000900DA49F800D911D11240895B7FF0C9432
:105B30008B2D0E948B2D821B930B0895DB018F937D
:105B40009F930E948B2DBF91AF91A29F800D911DBD
:105B5000A39F900DB29F900D1124089597FB072EDF
:105B600016F4009407D077FD09D00E94402E07FC60
:105B700005D03EF4909581959F4F0895709561955D
:105B80007F4F0895A1E21A2EAA1BBB1BFD010DC079
:105B9000AA1FBB1FEE1FFF1FA217B307E407F507DD
:105BA00020F0A21BB30BE40BF50B661F771F881FB9
:105BB000991F1A9469F760957095809590959B014F
:105BC000AC01BD01CF010895052E97FB1EF4009492
:105BD0000E94FB2D57FD07D00E94C22D07FC03D069
:105BE0004EF40C94FB2D50954095309521953F4FE8
:105BF0004F4F5F4F089590958095709561957F4FB9
:105C00008F4F9F4F08952F923F924F925F926F92C6
:105C10007F928F929F92AF92BF92CF92DF92EF923C
:105C2000FF920F931F93CF93DF93CDB7DEB7CA1BBD
:105C3000DB0B0FB6F894DEBF0FBECDBF09942A88E8
:105C4000398848885F846E847D848C849B84AA8490
:105C5000B984C884DF80EE80FD800C811B81AA811D
:105C6000B981CE0FD11D0FB6F894DEBF0FBECDBFE8
:105C7000ED010895EE0FFF1F0590F491E02D0994BA
:105C8000AA1BBB1B51E107C0AA1FBB1FA617B70762
:105C900010F0A61BB70B881F991F5A95A9F780957E
:105CA0009095BC01CD0108958F929F92AF92BF92C3
:105CB000CF92DF92EF92FF92CF93DF93EC01688156
:105CC00079818A819B81611571058105910521F496
:105CD00064E279ED8BE597E02DE133EF41E050E0B0
:105CE0000E94E42D49015A019B01AC01A7EAB1E4ED
:105CF0000E948B2D6B017C01ACEEB4EFA5019401E9
:105D00000E94992DC60ED71EE81EF91EF7FE06C08A
:105D100081E0C81AD108E10880E8F80AC882D9826F
:105D2000EA82FB82C701B6019F77DF91CF91FF9096
:105D3000EF90DF90CF90BF90AF909F908F9008959D
:105D40000E94542E089586E091E00E94542E0895FA
:105D500060930601709307018093080190930901F5
:105D600008952F923F925F926F927F928F929F92AF
:105D7000AF92BF92CF92DF92EF92FF920F931F9359
:105D8000CF93DF938B01EA016115710521F0DB01EF
:105D90008C9311969C93209739F09E0122503109E3
:105DA0002332310508F0D8C07C016701BFEFCB1A60
:105DB000DB0A5601F7016080862D90E00E94E32FF8
:105DC000892B11F07601F1CFFDE26F120AC0570165
:105DD00082E0A80EB11CD70111966C9077247394C1
:105DE0000BC0BBE26B1207C05701E2E0AE0EB11C64
:105DF000D70111966C90712CCE018F7E892B89F47E
:105E0000B0E36B1237C0F50180818F7D8835D1F406
:105E10006180F2E0AF0EB11C872D8260782EC0E168
:105E2000D0E0CA30D10551F1C031D10521F0C830E0
:105E3000D10599F409C0CC24CA94DC2CEC2CAFE039
:105E4000FA2E22C0209769F7C8E0D0E0CC24CA948B
:105E5000DC2CEC2CFFE1FF2E17C06FEF7FEFCB01A6
:105E60009E01442737FD4095542F0E94C22D6901A1
:105E70007A010AC02097A9F6CAE0D0E0E9E9CE2E5F
:105E8000DC2CEC2CE9E1FE2EF50160E020E030E0B6
:105E9000A9014E01AA2497FCA094BA2C1F0170ED11
:105EA000572E560CA9E0A51570F48FEB860D8A319C
:105EB00018F499EC592E06C08FE9860D8A3148F501
:105EC00089EA582E560C852D90E08C179D070CF50D
:105ED0006F3FD9F0C216D306E406F50698F0C50167
:105EE000B4010E949E2D9B01AC01852D90E0A0E0A5
:105EF000B0E0280F391F4A1F5B1F281739074A07D0
:105F00005B0710F46FEF01C061E03196D1016C9036
:105F1000C5CF0115110551F0662311F0319703C06B
:105F200071FE04C03297D801ED93FC9370FE07C058
:105F300050954095309521953F4F4F4F5F4F67FFEC
:105F400010C082E290E090938B0680938A066FEFF8
:105F50007FEF8FEF9FEF07C060E070E080E090E0A0
:105F600002C0B901CA01DF91CF911F910F91FF903B
:105F7000EF90DF90CF90BF90AF909F908F907F90E9
:105F80006F905F903F902F900895FC01882799278C
:105F9000E89421912032E9F3293010F02E30C8F333
:105FA0002B3241F02D3239F4689404C00E9417302E
:105FB000820F911D219120532A30C0F31EF4909539
:105FC00081959F4F0895911150C0803219F08950EA
:105FD0008550D0F7089548EC53E00E94F02F0895C3
:105FE000FA01A191B081009719F41097E1F0CD0169
:105FF000DC01CD010D90002011F4C00113C0FB01A4
:106000002191222319F02015D9F7F3CFFB0121911B
:10601000201519F41E92119606C02223C1F70D9087
:106020000020A1F7D001FA01A193B08308957AE08E
:10603000979F902D879F802D910D11240895F99998
:10604000FECF92BD81BDF89A992780B50895262F7D
:10605000F999FECF1FBA92BD81BD20BD0FB6F8944D
:10606000FA9AF99A0FBE01960895992788270895FC
:04607000F894FFCFD2
:1060740000008C06200001000000FF000200020066
:1060840002000200020002000200020002000200FC
:106094000200020002000200020002802500000546
:1060A400400AA1204EA50020244EA52C2330C01266
:1060B40000001A400AA1204EA5001B1E27522C23C3
:1060C400308025000005400AA1204EA50020244E62
:1060D400A52C2330004B000006400AD0009D490047
:1060E4007B289D492C233000E1000005400A45012E
:1060F400D7DC03B81E0EBF00232E48E801008A40F7
:106104000A6001555502AD1E20000023C8015458F1
:106114002074696D656F75742100596573004E6F45
:10612400002C00386368004E2F41002C205B005D7A
:106134002028002900486F70206368616E6E656CCA
:10614400200020402000456E746572696E672061EE
:1061540064617074697665206368616E6E656C2035
:1061640073656C656374696F6E2C207069636B6909
:106174006E673A007363616E6E6572206D6F64655D
:10618400004E4F5420454E41424C45440053656EE9
:1061940064696E672073657474696E677320746FC5
:1061A4002052580A00526573657474696E672073CF
:1061B400657474696E6773206F6E2052580A0041CB
:1061C400626F727465642065646974730A00696E31
:1061D40076616C69642073656C656374696F6E00C5
:1061E4000D0A496E76616C696420696E707574205D
:1061F4002D206469736361726465642107005365CB
:106204007474696E677320736176656420746F209B
:10621400454550524F4D0A00526576657274656467
:106224002073657474696E67732066726F6D2045A0
:106234004550524F4D0A004C6F616465642066619D
:1062440063746F72792064656661756C74730A0097
:106254004B657920616E64206368616E6E656C7352
:106264002072616E646F6D697A65640A004F7065AF
:106274006E4C52536E672054582073746172746963
:106284006E672000206F6E20485720006D6F647584
:106294006C65206C6F636B65643F00342B3400388D
:1062A40000382B340031320031322B3400313600C7
:1062B40050504D0052535349005344410053434CF2
:1062C40000525844005458440041494E004C424541
:1062D40045500053504B54524D00534255530053B4
:1062E400554D44004C4C494E440000070B0C101112
:1062F4001500B7012B032F033103350338033D0386
:10630400B7014003440349034D03510355035903A3
:106314005D0363036A036F0374038D028D028D02B0
:106324008D02160A1322312900000000C42BC9294A
:086334006A2B972B7C2BB92B7F
:107E00000F92CDB7DEB7112484B714BE81FFF1D035
:107E100082E08093C00088E18093C10086E0809377
:107E2000C20080E18093C4008EE0CDD088249924E4
:107E3000CC24C394F5E0DF2EE1E1EE2E73E0F72EC3
:107E4000B6D0082F813479F4B2D08983C2D0898129
:107E5000823811F481E005C0813811F485E001C059
:107E600083E09ED09AC0823411F484E103C085344B
:107E700019F485E0B6D091C0853561F498D0082F0B
:107E800010E095D090E0982E8824802A912A880CC2
:107E9000991C82C0863521F484E0A3D080E0E1CF34
:107EA000843609F04CC083D082D0A82E80D0B82E62
:107EB00000E011E07CD0F80181938F01AE16D1F77C
:107EC00088D0FB2DF53489F4E0E0F1E00BC0F9999E
:107ED000FECF92BC81BC0894811C911C819180BD15
:107EE000FA9AF99AEA1598F358C08B2D863409F05E
:107EF00054C0F401F7BEE89507B600FCFDCFF401CD
:107F0000A0E0B1E02C9130E011968C91119790E0B7
:107F1000982F8827822B932B12960C01C7BEE895C9
:107F20001124329681E0A038B80761F7F401D7BE7A
:107F3000E89507B600FCFDCFE7BEE8952EC0843774
:107F4000F1F435D034D0182F32D0B82E42D0FB2DDA
:107F5000F63421F4F40105914F010CC0FB2DF534EA
:107F600049F4F999FECF92BC81BC0894811C911C04
:107F7000F89A00B5802F14D0115049F70EC08537FC
:107F800039F427D08EE10CD085E90AD08FE069CF93
:107F9000813511F488E017D01CD080E101D050CF9A
:107FA0009091C00095FFFCCF8093C600089580910A
:107FB000C00087FFFCCF8091C00084FD01C0A89560
:107FC0008091C6000895E0E6F0E098E19083808318
:107FD0000895EDDF803219F088E0F5DFFFCF84E10E
:107FE000DFCF1F93182FE3DF1150E9F7F2DF1F9166
:0E7FF0000895282E80E0E7DFEE27FF27099492
:027FFE0001057B
:0400000300007E007B
:00000001FF
